:100000000C94380018950000189500001895000011
:10001000189500001895000018950000189500002C
:10002000189500001895000018950000189500001C
:10003000189500001895000018950000189500000C
:10004000189500000C9407051895000018950000FD
:1000500018950000189500001895000018950000EC
:1000600018950000189500001895000018950000DC
:100070008FEF8DBFC8EDE0EC4E2E84E08EBFD4E054
:10008000F4E05F2EA89584B7082E877F84BF88E1AF
:10009000992781BD91BDEEEFF3E0A0E0B1E08827A4
:1000A0008D933197E9F783E389B980E080BD88E1DA
:1000B0008AB90E941A0766248FEF8ABB8FEF8BBB29
:1000C0008FEF87BB8FEF88BB80E084BB8FEF85BB52
:1000D0008FEF81BB8FEF82BB8EEF86B98FEF87B931
:1000E000ECEFF0E080E40E94680758E0C895802DAE
:1000F0000E94620731965A95C9F704C00102201682
:1001000019111111E0E2F1E088E40E94680758E05B
:10011000C895802D0E94620731965A95C9F704C090
:100120000C04060C04040E20E4E4F1E080E50E94D7
:10013000680758E0C895802D0E94620731965A954D
:10014000C9F704C007050720202020200E94FF06D1
:100150008CE00E9468070E94DA0884E083BF89B7B8
:10016000826089BF7894809107018B7F809307011B
:1001700080910701806880930701809107018F7D3E
:1001800080930701809107018F7E8093070180E0B3
:1001900080930401E8E2F2E10E94F2060E94FD066B
:1001A000EEE3F2E10E94F2060E94F906E4E5F2E1D4
:1001B0000E94F20680E00E9462070E94FB06E0E6D1
:1001C000F2E10E94F20681E00E946207ECE6F2E1B1
:1001D0000E94F206E1E0F0E0A0E0B1E091E00E94D0
:1001E000C308E2E0F0E0A1E0B1E091E00E94C308C2
:1001F000E3E0F0E0A2E0B1E091E00E94C308E4E0B7
:10020000F0E0A3E0B1E091E00E94C3088091070113
:10021000806280930701E2E0F0E00E9411070E94F3
:10022000FF06E6E7F2E10E94F20681E00E94620723
:10023000E0E8F2E10E94F2060E94FD06ECE8F2E13D
:100240000E94F2060E94F906E2EAF2E10E94F2063A
:100250000E94FB06E8EBF2E10E94F20682E00E94B7
:100260006207EEEBF2E10E94F2060E94880580919F
:1002700007018B7F809307010E94C1050E94D90668
:10028000A0E1B1E08C93809110018093110195E081
:10029000A1E1B1E00E94AE07A0E1B1E08C918F71C5
:1002A0008C9300911101013011F00C94620100EE69
:1002B00040911001040FA0E0B1E00C930E9488056A
:1002C0000E94C10500911101033011F00C947301DB
:1002D00002EF40911001040FA1E0B1E00C930E94E5
:1002E00088050E94C10500911101043011F00C94A1
:1002F000840102EF40911001040FA2E0B1E00C93E1
:100300000E9488050E94C10500911101053011F07D
:100310000C94B201A0E1B1E08C9180FBA3E0B1E0CC
:100320008C9180F98C93A0E1B1E08C9181FBA3E0EA
:10033000B1E08C9183F98C93A0E1B1E08C9182FBC8
:10034000A3E0B1E08C9184F98C93A0E1B1E08C91B1
:1003500083FBA3E0B1E08C9185F98C930E94880522
:100360000E94C10500911101063011F00C94CE01DC
:10037000009110010F3111F00C94C501809107011B
:100380008068809307010C94CE01809107018F77DC
:100390008093070180911001809304010091110165
:1003A000023011F00C94DE0180910701806280938D
:1003B000070180910701806180930701A7E0B1E008
:1003C0008C9181FB16F00C942903809107018D7F9D
:1003D0008093070103B30F3F81E009F480E08F931E
:1003E00043B300911601041781E009F080E09F916A
:1003F0008923882311F40C94BE02A5E1B1E08C910D
:100400008F5F8C9300911501023311F00C94BC02A4
:1004100080E080931501009116010F3711F00C94C4
:100420001E02009100010F3F10F00C941C02A0E08E
:10043000B1E08C918F5F8C930C94B302073F11F065
:100440000C94320200910001003E18F011F00C945F
:100450002B020C94300280910001815080930001A6
:100460000C94B3020F3E11F00C943E02A3E0B1E0F5
:100470008C9190E289278C930C94B3020E3F11F07B
:100480000C944A02A3E0B1E08C9191E089278C930F
:100490000C94B3020F3D11F00C945B020091020129
:1004A0000A3F10F00C945902A2E0B1E08C918F5FEA
:1004B0008C930C94B3020D3F11F00C946F020091D9
:1004C0000201023F18F011F00C9468020C946D02C6
:1004D000809102018150809302010C94B3020F3B82
:1004E00011F00C948002009101010B3F10F00C946C
:1004F0007E02A1E0B1E08C918F5F8C930C94B302EB
:100500000B3F11F00C94940200910101023F18F08E
:1005100011F00C948D020C94920280910101815093
:10052000809301010C94B302063F11F00C94B302C6
:1005300080EE8093000186EF8093010186EF809327
:1005400002018EEE80930301809107018068809301
:100550000701809107018062809307018091070164
:100560008061809307010E9488050E94C1058091E7
:1005700007018062809307010C94C502A6E1B1E0F7
:1005800083B38C938DE280931501A7E0B1E08C9149
:1005900083FB882780F9809580FBA7E0B1E08C91F0
:1005A00083F98C93A7E0B1E08C9183FB16F00C9457
:1005B000FE02A7E0B1E08C9185FB16F00C94FC02E2
:1005C000809107018F7D809307018FEF0E94E606DF
:1005D00031E0A0E0B1E00E94E10631E0A1E0B1E04D
:1005E0000E94E10631E0A2E0B1E00E94E10631E0C4
:1005F000A3E0B1E00E94E1060C942903A7E0B1E07A
:100600008C9184FB16F00C942903809107018F7E56
:1006100080930701A7E0B1E08C9187FB16F00C9462
:1006200016038FE1809305010C941A038091040155
:100630008093050131E0A5E0B1E00E94E10632E0DF
:10064000AFE1B1E00E94E10632E0A8E0B1E00E9433
:10065000E106A7E0B1E08C9180FB16F00C94E90470
:10066000809107018E7F80930701ACE1B1E08C910E
:1006700087FB882780F9809580FBACE1B1E08C9105
:1006800087F98C93F89482E0E5E20E94D307ACE10D
:10069000B1E08C9187FB16F00C9462036CEC82E065
:1006A000E5E2BB27A6E121E02A930E94FB0764E470
:1006B00082E0E5E2BB27A6E121E02A930E94FB0746
:1006C0000C94BC036CEC82E0E5E2BB27A6E121E0E0
:1006D0002A930E94FB076EEB82E0E5E2BB27A6E1CE
:1006E00021E02A930E94FB07BB27A6E182E0E5E216
:1006F00021E02A930E941D08ADE1B1E05C93BB2785
:10070000A6E182E0E5E221E02A930E941D08AEE125
:100720000E94A407AFE1B1E00D931C93AFE1B1E0EB
:100730000D911C91ADE1B1E04D915527040F151FAE
:10074000AFE1B1E00D931C93AFE1B1E00D911C91CD
:100750004AE050E00E94A407AFE1B1E00D931C9382
:10076000AFE1B1E00D911C9140E150E00E94BF0665
:10077000AFE1B1E04D935C93789483ED12E00E9479
:100780000E07AFE1B1E00D911C914AE050E00E94EC
:10079000BF06A1E2B1E04D935C93A1E2B1E00D91FF
:1007A0001C914AE050E00E94A407A5E2B1E00D933D
:1007B0001C93AFE1B1E00D911C91A5E2B1E04D9128
:1007C0005C91041B150BA3E2B1E00D931C93A8EA06
:1007D000B4E0E1E2F1E00E9450080E94EA06ECEC8D
:1007E000F2E10E94F206A8EAB4E0E3E2F1E00E943E
:1007F00050080E94EA0682E00E946207EEECF2E1F5
:100800000E94F206A7E0B1E08C9187FB16F00C94F1
:100810001D040091210145E00E94CA08A4E0B1E056
:100820000C9300910401093118F011F00C941A0492
:100830000C941D0489E180930401AAE0B1E00D91BC
:100840001C914AE050E00E94A407AAE0B1E00D9399
:100850001C93AAE0B1E00D911C91003157E21507FD
:1008600010F00C946704AAE0B1E08D919C91A8E08F
:10087000B1E08D939C93A8E0B1E00D911C91ACE0A8
:10088000B1E04D915C91040F151FA8E0B1E00D930C
:100890001C93A8E0B1E00D911C91AEE0B1E04D9148
:1008A0005C91040F151FA8E0B1E00D931C93ACE020
:1008B000B1E08D919C91AEE0B1E08D939C93AAE064
:1008C000B1E08D919C91ACE0B1E08D939C9380E080
:1008D00090E0AAE0B1E08D939C9380910701806144
:1008E0008093070183ED1CE00E940E07A8E0B1E0B1
:1008F0000D911C91083E53E0150710F00C948404F0
:10090000E2EDF2E10E94F206A8E0B1E00D911C9147
:10091000043650E0150710F00C949204E2EDF2E179
:100920000E94F206A8E0B1E00D911C910A3050E05F
:10093000150710F00C94A004E2EDF2E10E94F2061B
:10094000A8EAB4E0E8E0F1E00E9450080E94EA065C
:10095000A7E0B1E08C9182FB16F00C94E504A2E1D3
:10096000B1E08C918F5F8C9300911201053011F0F2
:100970000C94E30480E080931201809107018B7F47
:1009800080930701C498E1E0F0E0A0E0B1E091E0DD
:100990007BE70E94B208E2E0F0E0A1E0B1E091E084
:1009A0007BE70E94B208E3E0F0E0A2E0B1E091E072
:1009B0007BE70E94B208E4E0F0E0A3E0B1E091E060
:1009C0007BE70E94B2080C94E90480E08093120156
:1009D000C49A28990C94FE04A7E0B1E08C9186FBA0
:1009E00016F00C94FC04809107018F7B8093070123
:1009F000AAE0B1E00E9492060C94030580910701E1
:100A00008064809307010C943E01F894FFCF0F920D
:100A10001F922F923F924F925F927F92AF92BF921E
:100A20000F931F932F933F934F935F936F937F93F6
:100A30008F939F93AF93BF93CF93DF93EF93FF93E6
:100A40008FB78F9385E082BFA6E0B1E08C918F5F76
:100A50008C9300910601093111F00C94320580E06D
:100A6000809306014091040100910601041710F0E3
:100A70000C943D05399A0C943E05399880910701F4
:100A8000826080930701ABE1B1E08C918F5F8C9322
:100A900000911B010A3F11F00C94560580E08093F1
:100AA0001B01809107018160809307018F918FBFA7
:100AB000FF91EF91DF91CF91BF91AF919F918F9176
:100AC0007F916F915F914F913F912F911F910F9166
:100AD000BF90AF907F905F904F903F902F901F906E
:100AE0000F9018950E94DF0812E80E94F708A3E112
:100AF000B1E01C910E94F708A4E1B1E01C910E94B2
:100B0000F7080E94EE0881E090E00E9495070895A2
:100B1000C49B0C9493058091070184608093070126
:100B200080E08093120180E08093130180910001A6
:100B3000809314010E94720581E0809313018091DB
:100B40000001809314010E94720582E080931301DA
:100B500080910101809314010E94720583E08093CB
:100B6000130180910201809314010E94720588E0B4
:100B70008093130180910301809314010E947205F8
:100B80000895A0E0B1E00D91112740EE50E0041B64
:100B9000150BA7E1B1E00D931C93A7E1B1E00D9116
:100BA0001C9142E050E00E94A407A7E1B1E00D9340
:100BB0001C93A7E1B1E00D911C9148E350E0041BA8
:100BC000150BA7E1B1E00D931C9381E080931A010E
:100BD0000E944806A2E0B1E00D91112746EF50E0D7
:100BE000041B150BA7E1B1E00D931C93A7E1B1E045
:100BF0000D911C9143E050E00E94A407A7E1B1E0F1
:100C00000D931C9382E080931A010E944806A1E094
:100C1000B1E00D91112746EF50E0041B150BA7E141
:100C2000B1E00D931C93A7E1B1E00D911C9143E05D
:100C300050E00E94A407A7E1B1E00D931C9383E06C
:100C400080931A010E944806A3E0B1E08C9185FBD5
:100C5000882780F9809580FBA8E3B0E08C9181F92A
:100C60008C93A3E0B1E08C9180FBA8E3B0E08C9181
:100C700082F98C93A3E0B1E08C9180FB882780F906
:100C8000809580FBA8E3B0E08C9183F98C93089564
:100C90008BE080931901A7E1B1E00D911C9109301F
:100CA00050E015071CF011F00C9458060C945D06EA
:100CB00080911901815080931901A7E1B1E00D9154
:100CC0001C91003050E015070CF402C00C946D0626
:100CD00080911901815080931901A7E1B1E00D9134
:100CE0001C91073F5FEF15070CF402C00C947D06C2
:100CF00080911901815080931901AAE1B1E02C91F2
:100D0000A9E1B1E01C910E940407E2EDF2E10E942A
:100D1000F206A8EAB4E0E7E1F1E00E9458080E9478
:100D2000EA060895ED91FC91EF5FFF4FFC93EE937F
:100D3000089509D00E94A40700FC10D0089503D0A4
:100D40001ED001F8F9CF0024E89457FF02C009D063
:100D5000689400F80BD010F80124089502D009D04F
:100D60000895509540954F5F5F4F0895E89417FFA1
:100D70000895009510950F5F1F4F68940895352FC3
:100D8000242FE894452B11F468940895512F402F97
:100D90000027112780E1440F551F001F111F021B60
:100DA000130B416018F4020F131F4E7F8A9599F7B9
:100DB000089588275F9B089500C05F9BFECF8CB18C
:100DC00008958D9103D03A95E1F708955D9BFECF8C
:100DD0008CB90895A8EAB4E08D91882311F072D0FF
:100DE000FBCF08950E94B607802D11F06BD0FACF8B
:100DF000089584E96DC084ED6BC080EC69C081E02A
:100E000067D015D080E864C08FE7213039F08FEBD0
:100E1000223021F083E9233009F083ED810F0C9417
:100E2000680788EE93E081D03197D9F7089583E081
:100E300099277BC08AEF90E00E949507D59AD49AB3
:100E4000D39AD29AD19AD09AD89885E090E00E940D
:100E50009507D998DD98DC98DB9ADA9AD99AEF93BE
:100E6000FF93ECE8F1E00E948907FF91EF91D99898
:100E700059D0D99AEF93FF93ECE8F1E00E948907EB
:100E8000FF91EF91D9984ED0D99AEF93FF93ECE868
:100E9000F1E00E948907FF91EF91D99843D0DA9849
:100EA000D99AEF93FF93ECE8F1E00E948907FF9154
:100EB000EF91D99837D088E20BD08EE009D086E048
:100EC00007D00895D89A829505D004D02BD00895E4
:100ED000D898F9CF859510F4DA9A01C0DA988595FB
:100EE00010F4DB9A01C0DB98859510F4DC9A01C000
:100EF000DC98859510F4DD9A01C0DD98D99AEF93BE
:100F0000FF93ECE8F1E00E948907FF91EF91D998F7
:100F100008953197F1F70895689462F80895E89478
:100F200062F8089581E090E000C0EF93FF93EE2710
:100F3000E82BE92B31F0E0EAFFE03197F1F7019778
:100F4000D1F7FF91EF9108950F92B801469F80016C
:100F5000479F100D569F100D0F900895903029F067
:100F60008C9186959A95E9F78C930895C89531965A
:100F70000020089591E0882321F08894991F8A9594
:100F8000E9F7892F909508950181082B018312813B
:100F900019231283EF93FF93E4E1F0E00E948907A5
:100FA000FF91EF9108950E948F07FF270E94BA07D3
:100FB000EBDFEF93FF93ECE7F7E00E948907FF91E7
:100FC000EF91182B128309230183EF93FF93E4E140
:100FD000F1E00E948907FF91EF911081182311F031
:100FE0000E948C07EF93FF93E4E6F6E00E948907E6
:100FF000FF91EF9108950E94BA07FF2729915D9113
:1010000048E0C2DF579510F4182B1283EF93FF933B
:10101000E4EDF0E00E948907FF91EF91182B128315
:10102000EF93FF93E4E2F0E00E948907FF91EF91D4
:101030004A9539F72A9519F708950E94BA07FF27AC
:10104000299148E05527A0DF09230183EF93FF93FF
:10105000E0E2F0E00E948907FF91EF91889410810F
:10106000182309F008945795EF93FF93E8EDF0E00B
:101070000E948907FF91EF914A9529F75D932A9580
:1010800001F70895000F111F221F331F08950095C7
:101090001095209530950F5F1F4F2F4F3F4F0895AC
:1010A000019110810EC001911191219130810BC0ED
:1010B0000191108117FF05C03FEF2FEF04C00081A1
:1010C00011272227332737FF03C0E1DF8DE28D93FD
:1010D000CF93DF93CF92DF92EF92AA24BB24CC244C
:1010E000DD24EE2440E2CAE0DD2755E093E3888169
:1010F000890F87FD9F7083FD907F891B89935A9587
:10110000A9F7C0DFAA1CBB1CCC1CDD1CEE1C4A9539
:1011100051F7E894EFE0FF2782910ED0EB30E0F733
:101120001EF068948A2D0CD088278D93EF90DF9065
:10113000CF90DF91CF910895982F829501D0892F7C
:101140008F70805D26F0803309F4089568948D9344
:101150000895E199FECFEEBBFFBB3196089591E073
:1011600001C092E07B3751F47FB7F894F2DF8D91A4
:101170008DBBE29AE19A9A95C9F77FBF77270895C8
:1011800091E001C092E0E5DFE09A8DB38D939A95EE
:10119000D1F70895FF93881BF9E0001FFA9511F429
:1011A000FF910895881F841B18F4840F8894F5CF4D
:1011B0000894F3CF979896988F988E9808958E9A62
:1011C0008F9803D08E9801D08F9AEF93FF93E0E130
:1011D000F0E00E948907FF91EF9108958E9A8F9A0F
:1011E000F4DF8E98869BFECFF0DF8F98EECF0894C9
:1011F000111F01C0110F69F08E9A18F400008F982A
:1012000002C08F9A00C0E1DF8E98869BFECFDDDFA3
:10121000F1CF8E9A8F98D9DF8E98869BFECFE89477
:101220008799689462F8D1CF20577A6D61636E69AF
:1012300061637A202052532D323332200000202067
:101240002020576572736A613A20312E3033202096
:10125000202000004A616B7562204D6F726F0000A4
:1012600020202020204D69726F7300006177204696
:1012700069726C656A00506F7A696F6D2047000073
:101280006F73753A20202D3536644200546F6E79A5
:10129000205779736F6B69653A20202020306442B3
:1012A0000000546F6E79204E69736B69653A202097
:1012B00020202030644200002035372E33004320A8
:1012C000202020323335362072706D002E004320EE
:0412D00020002000DA
:00000001FF
